:100000000C94D9000C94EB000C94EB000C94EB00D6
:100010000C94EB000C94EB000C94EB000C94EB00B4
:100020000C94EB000C94EB000C94EB000C9482010C
:100030000C94C0010C94EB000C94EB000C94EB00BE
:100040000C94EB000C94EB000C94EB000C94EB0084
:100050000C94EB000C94EB000C94EB000C94EB0074
:100060000C94EB000C94EB000C94EB000C94EB0064
:100070000C94EB000C94EB000C94EB000C94EB0054
:100080000C94EB000C94EB000C94EB000C94EB0044
:100090000C94EB000C94EB0000010000D600120061
:1000A000020000E80022002200000A013B002100BB
:1000B00000FA000900030000450104010309044996
:1000C00001280203090473011E0303090493011CA0
:1000D000000001C116001201000200000010CDABAB
:1000E00001FA00010102030109022200010100C01E
:1000F0003209040000010300000009211101000180
:10010000223B000705830310000105010905A10139
:100110000901A100093009310932093309340935CF
:100120000936093709380939150026FF0075089581
:100130000A8102C005091901291015002501750160
:1001400095108102C00403090428035B004D00617F
:10015000006E007500660061006300740075007237
:100160000065007200200068006500720065005D97
:100170000000001E035B00500072006F00640075F9
:100180000063007400200068006500720065005D77
:100190000000001C035B00530065007200690061F1
:1001A000006C00200068006500720065005D0000C2
:1001B000000011241FBECFEFD2E0DEBFCDBF11E0A3
:1001C000A0E0B1E001C01D92A231B107E1F70E94A9
:1001D000ED000C9427050C940000AF92BF92CF92D3
:1001E000DF92EF92FF920F931F93DF93CF93CDB7E0
:1001F000DEB76A970FB6F894DEBF0FBECDBFCC2432
:10020000C3947E010894E11CF11C8E01035F1F4F13
:10021000F894CAB80E9463010E9469017894F701BA
:100220001192E017F107E1F70E949303882381F709
:1002300060E80E94A10481E060E80E94A1047DE0E2
:10024000C72ED12CCC0EDD1E63E0B62E5AE3A52EB0
:10025000F894C6010E94D403882349F5D60180E0B2
:1002600090E02D913D91FC01EE0FFF1FED5FFE4FE1
:100270003183208301968730910599F7789482E045
:1002800061E00E94A104F8948091E900B092E90035
:100290009091E80095FF09C0F70191919093F100CA
:1002A000E017F107D1F7A092E8008093E900789475
:1002B000CFCF8091E80080FFFCCF08958091E800C7
:1002C00082FFFCCF0895E1E6F0E080E880831082B1
:1002D00008958FEF8093110180EA8093D8001092E7
:1002E000630086E089BD09B400FEFDCF80E88093FD
:1002F000D8001092E0008CE08093E20081E08093CF
:10030000110108951F920F920FB60F9211248F932F
:100310009F938091E1001092E10083FF0FC0109243
:10032000E90091E09093EB001092EC0092E1909341
:10033000ED0098E09093F0001092020182FF19C046
:10034000809111018230A9F4809100019091010106
:10035000009779F00197909301018093000183E069
:100360008093E9008091E80085FF03C08AE38093D1
:10037000E8009F918F910F900FBE0F901F901895DE
:100380001F920F920FB60F921124EF92FF920F93CC
:100390001F932F933F934F935F936F937F938F930D
:1003A0009F93AF93BF93CF93DF93EF93FF931092FD
:1003B000E9008091E80083FF3BC13091F10020917A
:1003C000F1000091F10010E04091F100942F80E0E5
:1003D000082B192B8091F100C82FD0E04091F1003B
:1003E000942F80E0C82BD92BE090F100FF2440919E
:1003F000F100942F80E0E82AF92A82EF8093E80048
:10040000263009F059C08FE990E09C01255030401A
:1004100004C081E28093EB000BC1FC01379745914A
:10042000549140175107D1F4F901459154914C175B
:100430005D07A1F42E5F3F4FF901859194912E5FE6
:100440003F4FF9012491A7014F3F510519F010F0DA
:100450004FEF50E0421750F4242F08C00796295F51
:100460003F4FF0E0873D9F07C1F6D3CFAEEF4091FD
:10047000E80050E0BA016570707061157105B9F35C
:1004800042FDD6C0322F213108F030E1AC01632F9C
:1004900007C0FA014F5F5F4FE491E093F1006150B4
:1004A0006623B9F7830F911D231BA093E800222335
:1004B000F1F63031E1F2BCC0253049F48EEF809383
:1004C000E8000E94590100680093E300B1C02930A0
:1004D00051F5332309F081C0009302018EEF809320
:1004E000E80041E080ED90E04093E900FC010196D6
:1004F000E491E093EB00EE2369F09C012F5F3F4F06
:10050000FC0184918093EC00C9010196F9012491CA
:100510002093ED004F5F453039F78EE18093EA007C
:100520001092EA0085C0283041F4303809F055C0F7
:100530000E945901809102015EC0222329F40E9489
:1005400059011092F1005EC0233AF9F48091E8005D
:1005500090E09C012570307021153105B9F382FDC2
:1005600067C080E090E0FC01EE0FFF1FED5FFE4FE3
:10057000208131813093F100208131812093F1007D
:1005800001968730910579F750C0243A91F4809113
:10059000E80090E09C012570307021153105B9F319
:1005A00082FD46C08C2FC7FF40C08F770E94BC04DD
:1005B00022C0253A91F40E945E0131E0E316F10475
:1005C00061F58C2F8F776091F100C7FF03C00E9407
:1005D000A10423C00E94E40420C0209749F5313AC9
:1005E000A1F4213019F40E9459011FC0223031F4C6
:1005F0000E94590181E08093F10017C02330C1F4BB
:100600000E9459011092F10010C0313289F4293052
:1006100041F40E945E018091F1008BEF8093E8002D
:1006200004C02A3011F02B3019F48EEF8093E800CB
:10063000FF91EF91DF91CF91BF91AF919F918F91FA
:100640007F916F915F914F913F912F911F910F91EA
:10065000FF90EF900F900FBE0F901F901895559A36
:1006600085E08A95F1F70000569A089598E025E014
:100670002A95F1F7000087FF02C0559801C0559AEE
:1006800025E02A95F1F7000056982AE02A95F1F71F
:1006900000C0569A915011F0880FE9CF55988AE022
:1006A0008A95F1F700C056982AE02A95F1F700C024
:1006B00099B1569A85E08A95F1F7000081E095FF9F
:1006C00080E008959C01559898E080E045E04A95C7
:1006D000F1F7000056984AE04A95F1F700C0880FFC
:1006E0004D99816045E04A95F1F70000569A915086
:1006F00069F72115310509F4559A95E09A95F1F7B6
:100700000000569840E14A95F1F7569A95E09A957F
:10071000F1F7000055980895569885E08A95F1F70D
:100720000000559808958BB18F798BB98AB18F7974
:100730008AB98FEF91EEA4E081509040A040E1F79C
:1007400000C000000E942F0382E30E94360388232A
:1007500021F00E948C0381E0089580E20E9436031C
:1007600087E70E9436030E948C039AE09A95F1F77E
:1007700000C00E942F038CE30E943603882321F0DF
:100780000E948C0382E0089580E00E9436038CE989
:100790000E94360380E20E94360380E00E94360306
:1007A0000E948C0380E008950F931F93CF93DF93F3
:1007B000EC010E942F0382E30E94360388EA0E9424
:1007C00036030E948C038AE08A95F1F700C00E94EC
:1007D0002F0383E30E94360380E090E00E946203CF
:1007E000082F10E01983088380E090E00E946203E4
:1007F000382F20E0022B132B1983088380E090E030
:100800000E946203082F10E01B830A8380E090E0BF
:100810000E946203382F20E0022B132B1B830A83D4
:1008200080E090E00E946203082F10E01D830C839B
:1008300081E090E00E946203382F20E0022B132B0E
:100840001D830C830E948C038AE08A95F1F700C017
:100850000E942F038CE30E94360383E80E94360334
:100860000E948C038AE08A95F1F700C00E942F0352
:100870008DE30E94360380E090E00E946203182F0F
:1008800000E01F830E8380E090E00E94620390E00E
:10089000802B912B9F838E8380E090E00E946203E7
:1008A000182F00E01987088780E090E00E9462031B
:1008B00090E0802B912B9987888780E090E00E94C0
:1008C0006203182F00E01B870A8781E090E00E94F6
:1008D000620390E0802B912B9B878A870E948C0378
:1008E0008AE08A95F1F700C00E942F038CE30E94F2
:1008F000360381EB0E9436030E948C038AE08A95BE
:10090000F1F700C00E942F038DE30E94360380E0C0
:1009100090E00E946203182F00E01D870C8781E0A1
:1009200090E00E94620390E0802B912B9D878C8742
:100930000E948C0380E090E0DF91CF911F910F9196
:1009400008951F93DF93CF930F92CDB7DEB7182F83
:1009500069830E942F038CE30E943603812F0E943B
:1009600036036981862F0E9436030E948C030F9004
:10097000CF91DF911F9108951F93DF93CF930F9233
:10098000CDB7DEB7182F0E942F038CE30E943603E9
:10099000812F80680E9436030E948C038AE08A952A
:1009A000F1F700C00E942F038DE30E94360381E01F
:1009B00090E00E94620389830E948C0389810F90DA
:1009C000CF91DF911F9108951F93DF93CF930F92E3
:1009D000CDB7DEB7182F69830E942F0382E30E94F0
:1009E0003603812F0E9436036981862F0E943603C9
:1009F0000E948C030F90CF91DF911F9108951F9358
:100A0000DF93CF930F92CDB7DEB7182F0E942F033D
:100A100082E30E943603812F80680E9436030E9481
:100A20008C038AE08A95F1F700C00E942F038DE3C2
:100A30000E94360381E090E00E94620389830E9455
:100A40008C0389810F90CF91DF911F910895F894C5
:020A5000FFCFD6
:00000001FF
